:020000040000FA
:02000000602876
:080008008610241C8614C000C0
:10001000030EC10083120513251B2428861F1628F2
:100020002208A400241C86142418861006181628FA
:100030000F30A9008B100314061F0310A40C410EEF
:100040008300C00E400E0900861B2C282208A40045
:10005000241C861424188610061C2C280F30A90096
:100060008B100314061B0310A40C410E8300C00E5A
:04007000400E090035
:1000C000A001A101A201A401A501AA01A601A70105
:1000D000A801A80AA901B101B201B301B401B50197
:1000E000B601B701B801C001C1018316FF30850018
:1000F000860086108312851B2514851F2510831604
:1001000085138312AA102A10051F2A14051BAA148E
:100110002A1C8D288316051383128501860107305A
:100120009F00C7308316810083127E3092007D309D
:10013000831692008312003083168C008312903055
:100140008B00A20BA12864000B19CF20B02025182A
:10015000AB28061EA3282A18DC20AA188D21A32864
:10016000A90803190800A803031D08001E30A800F1
:10017000861FC728A60A031D08002513A517A60178
:10018000A7018B138316011383128B170800A70A8C
:10019000031D08002513A517A601A70108000B11D0
:1001A000A9080319D8288513251C8517A903080059
:1001B00005098039850008008C1C08008C10051783
:1001C000000000000000000000000000000000002F
:1001D0000000000000000000000000000000050812
:1001E000A0000608A10005132019FB289630B102D3
:1001F000031C042907299630B10703180029072991
:10020000FF30B10022140729B10122100729A019DB
:100210000E299630B202031C17291A299630B2070C
:10022000031813291A29FF30B200A2141A29B201A7
:10023000A2101A29211921299630B302031C2A2958
:100240002D299630B307031826292D29FF30B30036
:1002500022152D29B30122112D29A11934299630F7
:10026000B402031C3D2940299630B40703183929EC
:100270004029FF30B400A2154029B401A211402941
:10028000A01847299630B502031C502953299630EF
:10029000B50703184C295329FF30B50022165329FE
:1002A000B5012212532920185A299630B602031C90
:1002B000632966299630B60703185F296629FF303F
:1002C000B600A2166629B601A2126629A11A6D29E6
:1002D0009630B702031C762979299630B7070318A0
:1002E00072297929FF30B70022177929B701221323
:1002F0007929201A80299630B802031C89298C2973
:100300009630B807031885298C29FF30B800A2174A
:100310008C29B801A2138C2908008C100508A000B4
:100320000608A100201A99290130B10703189E2957
:10033000A5290130B102031CA229A529FF30B10073
:100340002214A529B1012210A529A11AAC29013036
:10035000B2070318B129B8290130B202031CB5292C
:10036000B829FF30B200A214B829B201A210B829EE
:10037000A119BF290130B3070318C429CB290130C3
:10038000B302031CC829CB29FF30B3002215CB29A7
:10039000B3012211CB292119D2290130B407031846
:1003A000D729DE290130B402031CDB29DE29FF3006
:1003B000B400A215DE29B401A211DE29A019E52995
:1003C0000130B5070318EA29F1290130B502031CF1
:1003D000EE29F129FF30B5002216F129B5012212CC
:1003E000F1292019F8290130B6070318FD29042A3C
:1003F0000130B602031C012A042AFF30B600A216FF
:10040000042AB601A212042A20180B2A0130B707C9
:100410000318102A172A0130B702031C142A172ABE
:10042000FF30B7002217172AB7012213172AA01886
:100430001E2A0130B8070318232A2A2A0130B802DD
:10044000031C272A2A2AFF30B800A2172A2AB8013B
:06045000A2132A2A080095
:084000000000040000000000B4
:02400E00543F1D
:00000001FF
